:10000000020D27021004E4782DF22202100C78452C
:10001000E2FF22021014E47845F22202101C020CC6
:0E002000A42222021024220100000002102C53
:0300330002103484
:03003B0002103C74
:06004300207F4002104482
:03004B0002104C54
:0300530002105444
:03005B0002105C34
:0300630002106424
:03006B0002106C14
:0300730002107404
:03007B0002107CF4
:100083000210840204A6E59620E7FB75960EE4F5BC
:1000930097E59620E7FB759691E59620E7FB7814A4
:1000A300E597F2782CE2B40511E59620E7FBE4F539
:1000B300967823E2F597E4782CF27814E2FF30E2A5
:1000C3000FE59620E7FB759611E4F597782CF2225D
:1000D300EF30E41AE59620E7FB759611759708E56E
:1000E3009620E7FB759611759780E4782CF2782CAF
:1000F300E2600221B47814E220E00221B47BFE7AAC
:100103000079207D087C007F20120A947823E2FE88
:1001130018E27C0012057A782512057678271205F5
:10012300767820E2547F6421703108E21470022152
:10013300B414601314601A24F960111460182402B3
:10014300706C120BAE806A1200218065120CE38082
:1001530060120022805B12002680567821E2B40CE4
:1001630000504B90016C25E0732184218921B1213A
:100173008E21B12193219821B1219D21A221A72173
:10018300AC1205D8802B12080080261206DD8021D0
:10019300120A0A801C12028480171208CF801212DE
:1001A3000663800D120A518008120B7A8003120C29
:1001B3006D782CE2640170577814E220E151E596E2
:1001C30020E7FB759691E59620E7FB7814E597F217
:1001D300E230E40320E0387814740212059C400BEB
:1001E3001205A81207C112054A800912058D1207CC
:1001F300C112056B1205B4B5070818E2B506031260
:10020300056BE59620E7FB7596117814E2F5977870
:100213002CE26402706AE59620E7FB759691E596F9
:1002230020E7FB7814E597F2E230E05474401205BE
:100233009C400B1205A8120A9412054A8009120564
:100243008D120A9412056B1205B4B5070818E2B5AE
:10025300060312056B782CE270127821E2B4090CC4
:10026300781D120E14120DB6FF120B0B782CE264DC
:10027300046005E59620E7FB7596117814E2F5977F
:10028300227822E224DF7002612F14700261462477
:1002930021B40500400261529002A525E0500205F9
:1002A300837341AF41BB41DA41F161037A0E799522
:1002B30012094B900E9580447A0E79A712094B9040
:1002C3000EAAE493FE900EA9E4937C002400782BFD
:1002D300F2EC3E18F2807B7823E275F003A4243815
:1002E300F8120E14781D120E2D120DB6804E7BFFE0
:1002F3007A0E79B0781D120E2D900EB0E493803CE7
:100303007823E2FF64817047EF7BFFB4810E7A0E9E
:1003130079C2781D120E2D900EC2800C7A0E79C907
:10032300781D120E2D900EC9E49380107BFF7A0E78
:1003330079B9781D120E2D900EB9E493FFE41209DA
:1003430057800F7A0E79D01209377426F280031280
:100353000C6D7822E2FF64016013EF6402600EEF1C
:1003630064036009EF64046004EFB405177827E2BF
:10037300FFD3782BE29F18E2940040087826E270BE
:1003830003120952782CE264046008E59620E7FB27
:1003930012092122780074FFF2E47807F2120C6646
:1003A3002401120C5424FE604314604A24026002A8
:1003B300816C900113E0FEA3E0FF120C662403F9A5
:1003C300E43AFAC003C002C001120C4CFD780DE4FC
:1003D300F208EDF2D001D002D003120971120C4CD5
:1003E300FF900113E48FF0120DE18170780774011F
:1003F300F2120C5B8077120C662402F9E43AFA7865
:1004030018120E2D781B7404F27BFE7A0079011208
:100413000C2678057410F2087401F27801120E08A4
:10042300EF2401FFEE3410FEE43DFDE43CFCC00488
:10043300C005C006C0077805E2FE08E2FFE4F8F94C
:10044300AA06AB07D007D006D005D004C3120DF718
:10045300501B7805E2FE08E2FF120BFF7806E22448
:1004630000F218E23402F280B2E47800F2900090D5
:100473007461F0A37403F07800E2A3F07B017A00C7
:1004830079907847120E2DE92401120C547846F224
:100493007F611207507807E26008C27FE4F5D71244
:1004A300100122C0E0C0F0C083C082C0D075D0006C
:1004B300C000C001C002C003C004C005C006C0071D
:1004C300E59620E7FB759686E59620E7FB7811E530
:1004D30097F2E59620E7FB759682E59620E7FB7891
:1004E30012E597F2E59620E7FB759684E59620E7FB
:1004F300FB7813E597F27811E230E103120D0C78E3
:1005030011E230E203120C897812E230E0031200A8
:10051300897812E230E1031200067813E230E10336
:1005230012086D7811E230E003120D15D007D006E2
:10053300D005D004D003D002D001D000D0D0D082D7
:10054300D083D0F0D0E032781FE22440F218E234B6
:1005530000F2782BE224C0F218E234FFF218E2240E
:1005630040F218E23400F2227814E24408F2E4780C
:100573002CF222E2FE18E2240008F2EC3E18F222EA
:10058300120E14E92FF9EA3EFA22782AE2FC08E275
:10059300FD781D120E147F2022F2C3782BE29440C3
:1005A30018E2940022781D120E147D407C007F20F7
:1005B300227826E2FE08E2FF7829E222E2FD7C00AF
:1005C30008120E147F2122ECF208EDF24C22D3E242
:1005D3009F18E29E227822E2700F08E2700B7826C1
:1005E300E2700608E264026003120C6D7820E224D4
:1005F3007F6012146028240270537824E2704E083E
:10060300E260138048781CE2B404097824E27004A1
:1006130008E2600280377BFF7A0079298025781C05
:10062300E2B404057824E2600280227825E2B481F2
:100633001A782DE27BFFB403067A00792780047AC7
:100643000079291209397402F280058000120C6DB9
:10065300782CE264046008E59620E7FB1209212266
:10066300781CE2640260227820E2701D7824E27034
:100673001808E2701408E2701008E2700C7822E2A5
:10068300700708E2D394014005120C6D803C782377
:10069300E2D39400402C781C7404F2E4782DF2E544
:1006A3009620E7FB12096AE59620E7FB759612751B
:1006B3009704E59620E7FB75960EE4F5971200067E
:1006C3008008781C7403F2782DF2782CE2640460BD
:1006D30008E59620E7FB12094422781CE2640470C3
:1006E300567820E2FF60506401604C7822E2704744
:1006F3007824E270427826E2703D08E26002803797
:100703007820E2640270307823E2702B7825E2FFD0
:1007130064816005EF6402701EEFB4811DE59620CD
:10072300E7FB12096AE59620E7FB759611759710AA
:10073300782D7403F28003120C6DE59620E7FB120B
:10074300095E6008E59620E7FB12094422A2AF92F6
:1007530000C2AFE59620E7FB75960E759701E59607
:1007630020E7FB759691E59620E7FBAF97782DE29E
:10077300FEB4030DE59620E7FB759611759710807F
:1007830038EE7035782D04F2EF30E50BE59620E76F
:10079300FB759611759740EF30E20BE59620E7FB6A
:1007A300759611E4F59778461205BF120AD0E596BF
:1007B30020E7FB759611759701A20092AF22781579
:1007C300EFF27818120E2D78161205CA602DE596F1
:1007D30020E7FB7815E2F596E4FFFED37817E29F56
:1007E30018E29E40167818120583120DB6F597E5A8
:0C07F3009620E7FB0FBF00010E80E02203
:10080000781CE2640470507820E2FF604A64016062
:10081000467822E270417824E2703C7826E2703714
:1008200008E2600280317820E26402702A7823E2D4
:1008300070257825E2FF6481701DEFB4811CE59678
:1008400020E7FB12096AE59620E7FB75961175977C
:1008500040E4782DF28003120C6DE59620E7FB1240
:10086000095E6008E59620E7FB12094422E478144B
:10087000F2E59620E7FB75960E759701E59620E761
:10088000FB759694E59620E7FBAF97782DE2B403CD
:100890000CE59620E7FB75961475972022EF30E65D
:1008A0000BE59620E7FB759614759780120CD278AD
:1008B000411205BF120A947842120E14120DB6FFAF
:1008C000120B0BE59620E7FB759614E4F59722785A
:1008D00020E26480701B7822E2701608E270120831
:1008E000E2700E08E2700A08E2700608E264016035
:1008F00005120C6D801B781CE2FFB4040B7BFF7AA1
:1009000000792712093904F2EFB403051209330400
:10091000F2782CE264046008E59620E7FB120921D6
:10092000227596117597407401782CF2E47828F2BC
:1009300008F2227A0079297BFF781D120E2D782A81
:10094000E4F20822759611759748227BFF781D0204
:100950000E2DE2FF08E2CF782AF208EFF222759618
:100960000EE4F597782CE264042275960E759701D3
:1009700022780A120E2D7808EEF208EFF2780FEEC8
:10098000F208EFF2780DE2FE08E2FF7809E22FFDAF
:1009900018E23EFC780FE2FE08E2FFC39DEE9C5099
:1009A0001D780AE475F001120E1D120DB6FD120B32
:1009B000D87810E22401F218E23400F280C622E571
:1009C0009620E7FB759601759708E59620E7FB757D
:1009D0009607759707E59620E7FB759609759707C3
:1009E000E59620E7FB75960B75970775D7E0E596BA
:1009F00020E7FB75960F75978043E602D2AFE59628
:100A000020E7FB759601759701227820E2701B782C
:100A100024E2701608E2701208E2700E08E2700A12
:100A20007822E2700508E230E703120C6D782C742E
:100A300005F27823E2781C60057403F280037402E7
:100A4000F2782CE264046008E59620E7FB12094482
:100A500022781CE2640470227820E26481701B78A2
:100A600022E2701608E2701208E2700E08E2700AC4
:100A700008E2700608E264016005120C6D80051240
:100A8000093304F2782CE264046008E59620E7FB61
:100A9000120921227815EFF27818120E2D7816120D
:100AA00005CA602B7815E2F5964396C0E4FFFE7800
:100AB000171205D14016E59620E7FB78181205833A
:100AC000E597120DCF0FBF00010E80E3E4F59622EB
:100AD0007808EFF2780B120E2D78091205CA602AF9
:100AE000E59620E7FB7808E2F596E4FFFE780A1227
:100AF00005D14016780B120583120DB6F597E596D1
:100B000020E7FB0FBF00010E80E3227845E270353D
:100B10007842120E14120DB6B4552A78457401F2BB
:100B20007842120E147818120E2DE92401F9E43AD5
:100B3000FA120DB6781BF27B017A0079D1120C26DD
:100B4000782F7401F222D27F120C5B7F007E10128C
:100B50000CBCBFAA05C27F12100112001ED2AF1238
:100B600009BF120016E4782FF2782FE260FB12031F
:100B700097E4782FF212001680EF7820E26401707B
:100B80001A7826E2701508E270117822E2700C08DB
:100B9000E2700808E2700408E26003120C6D782C21
:100BA000E264046008E59620E7FB12094422120C77
:100BB000D27842120E14781D120E2D782612095288
:100BC000782CE264046010E59620E7FB75961175B9
:100BD0009740740212092922A2AF9200120D1E8EB4
:100BE000088F0975B7A575B7F1438F01120D2085E0
:100BF0000982850883EDF0538FFEA20092AF22A2F6
:100C0000AF9200120D1E8E088F0975B7A575B7F14A
:100C1000438F03120D20850982850883E4F0538FEA
:100C2000FCA20092AF227815120E2DE4FF781BE291
:100C3000FEEFC39E50157818120D02120DB6FE7805
:100C400015120D02EE120DCF0F80E2227842120E25
:100C500014E92402F9E43AFA020DB6900113741073
:100C6000F0A37401F0227842120E14E922E59620D6
:100C7000E7FB75960EE4F597E59620E7FB75961170
:100C8000759720782C7404F222781C7402F2E59691
:100C900020E7FB759601759701E4782CF208740340
:100CA000F208F22243B203E4F5B943B980120CF31F
:100CB00043B9C0120CF3E5B930E5FB22A2AF9200B4
:100CC000C2AF8E088F098F828E83E493FFA20092B9
:100CD000AF227B017A00794E7842120E2D78417452
:100CE0000AF222782CE264046008E59620E7FB1201
:100CF000094422E4FFFE0FBF00010EBE01F8BFF45D
:100D0000F522120E14E92FF9E43AFA227815E224BA
:100D100001120564227815E2240112056422C2AF93
:100D200075FF8075EF0222787FE4F6D8FD75812F7C
:100D300075D900020D71020B46E493A3F8E493A366
:100D40004003F68001F208DFF48029E493A3F8540D
:100D500007240CC8C333C4540F4420C8834004F490
:100D600056800146F6DFE4800B01020408102040A3
:100D700080900E36E47E019360BCA3FF543F30E5C3
:100D800009541FFEE493A360010ECF54C025E06018
:100D9000A840B8E493A3FAE493A3F8E493A3C8C5E6
:100DA00082C8CAC583CAF0A3C8C582C8CAC583CAD7
:100DB000DFE9DEE780BEBB010689828A83E022503C
:100DC00002E722BBFE02E32289828A83E49322BBEC
:100DD000010689828A83F0225002F722BBFE01F3CA
:100DE00022C5F0F8A3E028F0C5F0F8E5821582707E
:100DF000021583E038F022EB9FF5F0EA9E42F0E91D
:100E00009D42F0E89C45F022E2FC08E2FD08E2FE8B
:100E100008E2FF22E2FB08E2FA08E2F922FAE2FB2A
:100E20000808E2F925F0F218E2CA3AF222EBF208D9
:100E3000EAF208E9F2228830FFFFFFFFFFFFFFFF21
:100E40006040004E000000000000000000000000B4
:100E50000000000000000000000000000000000092
:100E60000000000000000000000000000000000082
:100E70000000000000000000000000000000000072
:100E8000000000008938FF0EF6FF0EFBFF0F2783DE
:100E90002C00030300120110010000004025130084
:100EA000000000010200010902290001010080AFD9
:100EB00009040000020300000009210101000122D1
:100EC00026000705810340000A0705020340000AC7
:100ED0000600FF0901A1018555953F750826FF0011
:100EE00015000901910285619502750826FF00151C
:100EF0000009018102C005030904002A036100758D
:100F000000730074007200690061006D0069006385
:100F10000072006F00730079007300740065006D4B
:100F2000007300200000002A03410053007800787D
:100F30000078002000550053004200200042006F5E
:100F4000006F0074006C006F006100640065007247
:030F50000000009E
:00000001FF
